:1000000054C0CDC16DC06CC06BC06AC069C068C04F
:1000100067C066C065C064C063C062C061C060C0C4
:100020005FC05EC05DC00403090418037200610074
:10003000700068006E00650074002E006E006500A0
:1000400074001A034A0061006700750061007200C5
:100050002000410074006100720069000A03310051
:1000600030003000300005010905A1010901A1009F
:1000700009300931150026FF00750895028102C07C
:100080000509190129111500250175019511810234
:10009000750195078103C01201010100000008816C
:1000A000177B050001010203010011241FBECFE5EB
:1000B000D4E0DEBFCDBF10E0A0E6B0E0E6E3FBE0B9
:1000C00002C005900D92AA39B107D9F710E0AAE94C
:1000D000B0E001C01D92AA3EB107E1F721D329C5C6
:1000E0008FCF85B7836085BF8BB780648BBF83EC70
:1000F0008093C00008950F931F93CF93DF93909147
:10010000D00019160CF0AFC02091CD008091CC002A
:100110008D3209F09EC08AE5809361009B3009F022
:1001200098C0CCE0D0E0C21BD109CC52DF4F88810F
:10013000807609F080C01092BE008981882359F42E
:100140001092BF008EEB90E09093CF008093CE0092
:1001500030E822E077C0853021F48A818093D10095
:1001600068C0863009F04AC08B81813009F441C0F3
:10017000823019F4CE0176D260C0833069F58A816D
:10018000882349F486E290E09093CF008093CE00DC
:1001900030EC24E057C0813049F48AE290E090933B
:1001A000CF008093CE0030EC28E14CC0823049F47F
:1001B00082E490E09093CF008093CE0030EC2AE16F
:1001C00041C08330E9F58CE590E09093CF008093B7
:1001D000CE0030EC2CE036C0813249F48DEA90E05C
:1001E0009093CF008093CE0030EC29E02BC0823278
:1001F00039F5CE0137D2282F30EC24C0883019F4DD
:1002000083ED90E00AC0893021F48A818093D30085
:1002100010C08A3049F48EEB90E09093CF00809329
:10022000CE0030E821E00EC08B3019F483EC8093CF
:10023000C00030E806C0CE0143D2282F30E802C00B
:1002400030EC20E08F81882339F48E81821728F0EA
:1002500003C030E880E001C0822F30939A00809381
:1002600060001092D0008091610084FF49C08091AD
:1002700060008F3F09F444C0182F893008F018E05F
:10028000811B8093600080919A0080FD02C00BE486
:1002900001C003EC8F5F80939A002091CE003091D3
:1002A000CF0086FD05C0D901912FE6EBF0E011C02B
:1002B000A6EBB0E080E090E006C0F901E80FF91F7E
:1002C000E491ED9301961817C1F705C08D918193C4
:1002D00091509923D9F7F901E10FF11DF093CF0067
:1002E000E093CE0086EB90E0612F55D0183019F0E6
:1002F0008FEF809360000093B5001C5F1093610046
:100300009AE080B3857031F49150D9F71092D10002
:100310001092CB00DF91CF911F910F9108951F9301
:10032000DC01162F8091620084FF0AC08091C0001A
:1003300098E889278093C000912FE1ECF0E007C096
:100340008AE580936200F8CF8D9181939150992333
:10035000D9F781EC90E0612F1ED01C5F10936200F2
:100360001F910895A82FB92F8FEF9FEF41E050EA1A
:10037000615070F02D9138E0722F7827969587950F
:10038000269570FF02C0842795273A95A9F7F0CFEC
:10039000809590950895E6DF8D939D930895CF9372
:1003A000CFB7CF93809BFECF809B09C0809B07C0B7
:1003B000809B05C0809B03C0809B01C09EC0DF93D3
:1003C000C091CD00DD27CC52DF4F809B02C0DF9172
:1003D000EBCF2F930F931F9300B32FEF00FB20F968
:1003E0004F933F9310B34FEF012700FB21F93BE000
:1003F00031C04E7F012F10B3216028C0102F4D7FD8
:100400002260000000B329C04B7F2460012F000050
:1004100010B32BC010B3477F28602AC04F7E00B3B3
:1004200020612CC04F7D10B320622FC04F7B00B3E2
:10043000206432C0422700B349934FEF00001027D9
:1004400010FB20F910B31570A9F1297F91F2012753
:1004500000FB21F900B3237F89F23150F0F110271E
:1004600010FB22F910B3277E79F2012700FB23F954
:100470002F7C81F200B3102710FB24F92F7971F241
:1004800000C010B3012700FB25F92F7359F200C0FB
:1004900000B3102710FB26F9223040F200C010B341
:1004A000012700FB27F9243028F64F77206810B386
:1004B0000000F9CF3B503195333010E41ABFB8F04B
:1004C000C31BD0400881033C41F10B3431F1198149
:1004D000412F1F772091CB00121731F4093691F18B
:1004E0000D3279F0013E69F022272093D2003F912E
:1004F0004F911F910F912F91DF91CF91CFBFCF914E
:1005000018950093D2003F914F911F910F912F9119
:10051000DF91CAB7C6FD46CFF0CF0091D2000023CD
:1005200031F31091D0001123A1F53430A2F13093B2
:10053000D0000093CC001091CD003BE0311B3093F4
:10054000CD0029C00091D00001301CF50AE547FD1F
:1005500009C03091610034FD20C000936100C5EBFB
:10056000D0E01FC03091620034FD17C000936200DC
:10057000C0ECD0E016C0052710E002BB1FC0052765
:1005800022C0052727C005272CC0052710E002BB85
:1005900033C04AE503C042ED01C0432FC4E1D0E0BF
:1005A00032E011B31560909A02B311BB5F9355E02E
:1005B00020E820FF052702BB279517951C3FD8F69A
:1005C00020FF0527279502BB17951C3FC0F620FF8B
:1005D00005272795179502BB1C3F98F620FF052796
:1005E000279517951C3F02BB70F600C0499120FF6C
:1005F000052702BB279517951C3F38F620FF0527D6
:10060000279502BB17951C3F38F520FF0527279536
:10061000179502BB1C3F10F520FF0527279517955E
:100620001C3F02BBE8F4242F3A9519F60A7F5F912C
:1006300002BB00C01091D100C651D04011F0109300
:10064000CB0010E41ABF016011B31A7F402F4A7F1C
:1006500002BB11BB42BB4BCF0527D3CF0527D8CF59
:100660000527DDCFFC018081807641F581818630D0
:1006700029F583818230D1F0823269F08130F1F442
:1006800080919F009091A0009093CF008093CE0026
:100690008091A100089580919C0090919D0090937D
:1006A000CF008093CE0080919E00089583E690E075
:1006B0009093CF008093CE0082E2089580E0089569
:1006C000FC0124EA30E03093CF002093CE008081FB
:1006D0008076803219F58181813079F4E091A20031
:1006E000F091A3000088F189E02DC9010995E091FE
:1006F000A200F091A30080810895823041F48AEA3B
:1007000090E09093CF008093CE0081E008958A30EE
:1007100029F483818093AA0080E0089580E0089501
:10072000CF92DF92EF92FF920F931F9386B399D0EF
:10073000FC019093A3008093A20084819581909303
:100740009D0080939C00828180939E00808591858E
:10075000009731F09093A00080939F00868107C09E
:1007600087E990E09093A00080939F00D2D180937E
:10077000A10080919E0080937C0014BA8FEF85BB0E
:1007800088EF82BB85E081BB11BA83BF8FE085BD56
:1007900084EC83BDE091A200F091A3000284F38574
:1007A000E02D09959EDC7894FF2401E010E0CC2434
:1007B000C39490E8D92E04C0FF24F39400E01E2DCA
:1007C000A89599DC002341F0E091A200F091A300EC
:1007D0000484F585E02D099508B600FE0EC0C8BE5C
:1007E000E090AA00EE2049F0153018F4FF24F394AD
:1007F00005C08BEFE82EE10E01C0E12E08B607FE22
:1008000016C0D8BEFF20A9F4E091A200F091A30089
:100810000484F585E02D0995E091A200F091A300F4
:100820000684F785E02D0995882319F4C7CFFF20AA
:1008300029F28091620084FFBFCFE091A200F09185
:10084000A3000088F189E02D84EA90E00995E09109
:10085000A200F091A30084EA90E0608160DDFF24B3
:10086000ADCF86E690E090938A008093890085E87A
:1008700090E00895009741F0DC01EBEAF0E085E0BC
:1008800001900D928150E1F7A0EBB0E0EBEAF0E0CF
:1008900085E001900D928150E1F7089580919700D5
:1008A00090919800892B31F0109298001092970047
:1008B00081E008958BEA90E060EB70E045E050E065
:1008C0002BD108950F931F93DF93CF93CDB7DEB74E
:1008D00067970FB6F894DEBF0FBECDBF80E88E835A
:1008E0008D831F82188619861A861B868CE0FE016E
:1008F0003C96DF011D928A95E9F7FE01319640E0B2
:1009000050E000E210E0A0E7B7E1C801042E02C009
:10091000959587950A94E2F7682F85B3362F309521
:10092000832385BB84B3862B84BBCD010197F1F76C
:1009300023B386B390E08873907095958795237064
:10094000282B2083B09B02C02062208384B33823ED
:1009500034BB85B3682B65BB4F5F5F4F3196443026
:10096000510599F68C81A82F8981E82FF0E08A81C2
:10097000682F70E08B81482F50E0A4FD02C08FEFFC
:100980008D83A3FF1D82A2FD02C08FEF8E83CF0156
:1009900004E0969587950A95E1F721E030E08227FB
:1009A000932781708E87CB0114E0969587951A95D1
:1009B000E1F78227932781708D87CA01B4E096956D
:1009C0008795BA95E1F78227932781708C87CF01AD
:1009D00003E0969587950A95E1F782279327817022
:1009E000898BCB0113E0969587951A95E1F78227BD
:1009F00093278170888BCA01B3E096958795BA9545
:100A0000E1F78227932781708F87CF01969587958D
:100A1000969587958227932781708C8BCB0196952D
:100A20008795969587958227932781708B8BCA012E
:100A300096958795969587958227932781708A8BBF
:100A4000CF01F5E096958795FA95E1F782279327F0
:100A500081708F8BCB0175E0969587957A95E1F73C
:100A60008227932781708E8BCA0155E096958795D2
:100A70005A95E1F78227932781708D8BA5FF1E82FF
:100A80009A2F9095917040FF926060FF9460E0FF14
:100A90009860A1FF90618C85811190628D85811194
:100AA00090648E8581119068FE013F9630E021E0D0
:100AB000AE01495E5F4F80818111322B220F31964A
:100AC000E417F507C1F72F89211121E08D8180936B
:100AD000AB008E818093AC009093AD003093AE005C
:100AE0002093AF0067960FB6F894DEBF0FBECDBF60
:100AF000CF91DF911F910F9108951F931FB7F89425
:100B000014BA8FEF85BB17BA88BBDCDE1FBF1F91FD
:100B1000089582E190E00895FB01DC0104C08D910D
:100B20000190801921F441505040C8F7881B990B5F
:060B30000895F894FFCFC8
:100B3600FF5A5A090222000101008032090400000E
:100B46000103000000092101010001220000070540
:100B5600810308000A050031000000000000007D46
:0A0B66000562044E043A0401000089
:00000001FF
